S00600004844521B
S1236000CEC00018CE6133C62918A600A7000818085AC10026F3CEC10018CE615CC629188B
S1236020A600A7000818085AC10026F3861ABDFFB8C604BD611E861ABD6127CE6185BDFF44
S1236040CAC602BD611E861DBD6127CE619FBDFFCAC602BD611E861BBD6127CE61B4BDFFA9
S1236060CAC602BD611E8618BD6127CE61CCBDFFCAC606BD611E8600B71009B61008840139
S1236080BD610BB7C00DB61008840244BD610BB7C015B6100884044444BD610BB7C01DB6B1
S12360A010088408444444BD610BB7C025B61008841044444444BD610BB7C10DB610088435
S12360C0204444444444BD610BB7C1158614BD6127CEC000BDFFCABD60F9BDFFC4BDFFC489
S12360E08614BD6127CEC100BDFFCABD60F9860BBDFFB8BDFFB87E607B18CE00408608BD4F
S1236100FFB81809188C000026F3394848484844444444840F8B3081392F028B0739BDFFBD
S1236120C45AC10026F839168620BDFFB85AC10026F83972656164696E67207377303A2015
S12361402020207377313A202020207377323A202020207377333A202020200472656164B9
S1236160696E67207377343A202020207377353A202020207377363A204E43207377373A86
S1236180204E432004506F727420442053776974636820492F4F2050726F6772616D047533
S12361A073696E6720746865204D3638484331314556420462792053746576656E204A2E18
S12361C020446F6D62726F77736B690452656E7373656C61657220506F6C79746563686E8C
S11061E0696320496E7374697475746504F5
S9030000FC
